:020000040800F2
:10500000B81A0020D5500008D9800008E97C0008B3
:105010000000000000000000000000000000000090
:10502000000000000000000000000000958A000859
:105030000000000000000000B98800087D8B000817
:10504000E7500008E7500008E7500008E750000864
:10505000E75000084D5C0008E7500008E7500008E2
:1050600000000000E7500008895B0008E7500008D6
:10507000E7500008257E000800000000E750000807
:1050800000000000E75000080000000000000000E1
:10509000E750000800000000E7500008E750000853
:1050A000E7500008E7500008E7500008BD920008EC
:1050B000E7500008E7500008000000000000000072
:1050C0000348854600F08AFC004800478DA0000890
:1050D000B81A00200448804704480047FEE7FEE76E
:1050E000FEE7FEE7FEE7FEE7198C0008C150000866
:1050F00030B50B46014600202022012409E00D4670
:10510000D5409D4205D31D469540491B25469540F7
:1051100040191546521E002DF1DC30BDF0B51FB40C
:105120000646002082B005464024019100901BE015
:10513000019922460F46304600F078FB049A059B01
:10514000801A994110D310461946224600F05EFBA2
:10515000361A8F410197224601200021009F00F05E
:1051600055FB38184D4100902046641E0028DFDCB6
:10517000019B00982946324607B0F0BD03460B4319
:105180009B0703D009E008C9121F08C0042AFAD2FD
:1051900003E00B780370401C491C521EF9D2704783
:1051A000D2B201E00270401C491EFBD270470022BF
:1051B000F6E710B513460A4604461946FFF7F0FF16
:1051C000204610BD30B504460020034600E05B1CBD
:1051D000934203D2E05CCD5C401BF8D030BDF8B503
:1051E00002464A40D40F42004B0052085B089A42E4
:1051F00002D20246084611464A0023D0C30D4A0097
:10520000DDB2120EAD1A202D35DA49020126490A07
:10521000F6058A19002C00D0524220214F1B11465E
:10522000B9402A411018C20D9A4221D0002C17D043
:10523000012D08DCDA05801AD20F8019D207DBB203
:1052400000F020FBF8BDDA05801A012340001B06A0
:10525000C01880185A428018CA0F1043490007E04E
:105260004908C2071143DA05801A801940088018DE
:1052700000F000FBF8BD61000122511A001BF7E7A6
:105280000122D2075140AAE70122D2075040A6E7E7
:10529000024670B54A40D30FDB0740002DD04A00CC
:1052A0002AD0010E140E000212020919400A520AF5
:1052B0008418E50104465443000A120A2E045043A0
:1052C000A4194219200CC543AA18120C0125AD03DC
:1052D000521C521912047F39240400D0521C10436E
:1052E00001D44000491EC2B20C06C0092018401C5F
:1052F0004008802A02D003E0002070BD4008400032
:10530000002900DA0020184370BD70B502464A40FB
:10531000D50F40004A00ED0740085208002814D07D
:10532000002A12D0C40DD30D41020120C005520243
:10533000490A520AE41A091812187D34914201D31D
:10534000641C00E04900002C01DA002070BD00233D
:10535000914201D3891A0343400849000028F7D13C
:1053600000290AD0914202D10121C90705E09142EA
:1053700001D2012101E00121C943E005C018401913
:1053800000F078FA70BD0000F0B5074608465840B6
:1053900087B0C00F049048000E46590040084908E5
:1053A000BC1A884105D2384631461E4617460B4680
:1053B00002465800400810434CD0300D0390400581
:1053C0005900400D490D0590401A0290402872DAAC
:1053D00018030121000B090508430190049800926D
:1053E000002805D001995242002088410092019086
:1053F000029840210A1A0199009800F007FA054620
:105400000C466B4607CB00F022FAC0197141039A93
:105410000E0D0023D71756401A467A40164344D043
:10542000049A002A2DD0029A012A039A15DC12054B
:10543000C01A914101263605001C7141D20F059E0C
:10544000D2070093019202962A46234600F060FAA2
:1054500007B0F0BD38463146FAE71605224A0F4636
:10546000B218C01AB74101210905001C4F410018AC
:105470007F41114618187941E20F10436D196441BC
:1054800013E0E2076D0815436408C2071443039A4A
:1054900001261205C01A91413605001C7141CE0744
:1054A000400830434908C01851412A46234600F0BD
:1054B00022FACDE7FFE7049801224000C117121A33
:1054C00000238B4104983146C417381AA141EEE7F6
:1054D00030B40124E407634030BC55E730B4012404
:1054E000E407614030BC4FE70000E0FFF0B51FB4B7
:1054F00088B00B990998002448400999C00F4900C9
:1055000049080991C0070B990090490049080B917F
:1055100009990898A64608431CD00B990A98084395
:1055200018D0099801244000420D4800410D099807
:1055300024050003000B204309900B980003000B87
:1055400020430B9050181C4940180022019014462B
:10555000104605E0002001460DB0F0BD032801DA39
:10556000034600E003239C46C11A0AAE0AE05F002E
:1055700008ADED5B4F00F75B7D430027AA187C4127
:10558000491C5B1E6145F2DD410004AB5A52210407
:10559000120C0A43240C401C0828DFDB01980290FF
:1055A0000099704601910090059B049A079906980E
:1055B00000F0AEF9D0E700000DFCFFFFF0B50C469F
:1055C0005C4085B0E40FE40703944C0000266408B7
:1055D00059009446490802460296224321D0624669
:1055E0000A431ED06200570D4A000E032303550DD7
:1055F000012402462C492405781B1B0B360B40184E
:1056000023432643614600901C46501AB44103D3FD
:105610000098401C009002E0921800985B4100281E
:1056200003DA0020014605B0F0BD00200121090584
:105630000746864611E064461D46141BB54106D355
:105640006546521BB341744607430C43A646CD073B
:1056500040084908284392185B4105460D43EAD1AA
:105660001046184313D06046194650407140084315
:1056700006D06046101AB34106D20122002306E08C
:1056800000220123DB0702E00122D24353100098DD
:1056900074460105381C6141029C039D0019694153
:1056A00000F029F9BFE70000FD03000010B500225B
:1056B0009623114600F0E6F810BD00000EB5C217A3
:1056C000C10F5040CA0740180021054B02930192B8
:1056D00000910A460B4600F01BF903B000BD000024
:1056E000330400000EB505490291002100910A46DD
:1056F0000B46019100F00CF903B000BD330400002B
:10570000410040020122400AD205090E80187F297B
:1057100001DA00207047962903DC9622511AC8400E
:10572000704796398840704770B5CD0F4A0009031D
:105730000123090B1B0519430B4BED070024520DE8
:105740009A4201DA002070BD074B34339A4203DCE1
:105750009A1A00F06BF802E00449511888402C4373
:10576000F1D0404270BD0000FF030000CDFBFFFF01
:105770004A0009030123090B1B051943094B10B506
:10578000520D9A4201DA002010BD064B34339A4282
:1057900003DC9A1A00F04AF810BD034951188840FA
:1057A00010BD0000FF030000CDFBFFFFC20FD207BA
:1057B000400040080BD0C10D0723DB01C91840028F
:1057C0000905400A1143C2084007114370470020F1
:1057D00001467047CB0FDB07490010B54908024668
:1057E0000A4307D00A0D07240903E401090B121B21
:1057F000002A01DC002010BDC900440F0C43C10089
:10580000E018D205801800F035F810BD10B5202A38
:1058100004DB0146203A9140002010BD9140202336
:105820009C1A0346E3401943904010BD10B5202A4E
:1058300004DB0846203AD040002110BD0B46D3407F
:10584000D0402024A21A91400843194610BD10B53B
:10585000202A06DBCB170846203A1041C1170B431C
:1058600006E00B461341D0402024A21A9140084381
:10587000194610BD002904DA401C490001D1400836
:105880004000704770B40024050C05D110240004BA
:1058900002D1002921D01124050E01D100020834C3
:1058A000050F01D10001241D850F01D18000A41C2A
:1058B000002801DB4000641C002908D020252E1B95
:1058C0000D46F540A14000D00121294308430106BF
:1058D0001B1B000ADB1D02D5002070BC7047DB05D6
:1058E000181880180029F8DA401C4900F5D170BC5E
:1058F00040084000704710B5002B08DA0024401C17
:10590000614192185B411A4301D14008400010BD2B
:10591000F0B51FB482B005460C0003D0084603F072
:105920008BFD02E003F088FD203002460090214606
:105930002846FFF76BFF049B059A04460F46184361
:105940001143084314D0184610431BD0009840213F
:105950000A1A18460599FFF769FF05460E46009A90
:1059600005990498FFF752FF084305D0012004E091
:105970002046394607B0F0BD0020C11705430E434D
:105980002C43374300990E986305401A7905E40AC1
:1059900000220C43FD0A0A3002D500200146E9E747
:1059A0000105101969410C9C0D9D00196941FFF713
:1059B000A2FFDFE710B5002904DB0124E407404221
:1059C0008C412146002B04DB1C460123DB0752429D
:1059D000A341994200D1904210BD0000064C012520
:1059E000064E05E0E36807CC2B430C3C9847103487
:1059F000B442F7D3FFF768FB5CA500087CA500085C
:105A000070B5044600688168490720D58168102672
:105A10004907002905DA8168890702D48168314382
:105A2000816001F047F905460DE001F043F9401BA4
:105A30000A2808D9606D30436065A06D01210843D4
:105A4000A065084670BD206880684007EDD400203E
:105A500070BD000038B50446064805490068FFF7E8
:105A600047FB604300E0401E00900028FBD138BD9A
:105A700040420F0010010020F8B50446006881681C
:105A80008907890F012925D10168C90722D08168BA
:105A9000052211401025012601290FD1816802221B
:105AA0001143816021680320086001F003F9074673
:105AB0000CE001F0FFF8C01B0A2807D9606D2843ED
:105AC0006065A06D3043A0650120F8BD2068806846
:105AD000C007EED10020F8BDF8B504460068816823
:105AE0008907890F012902D10168C90722D181687C
:105AF000114A10261140012500290ED18168294341
:105B000081600120FFF7A6FF01F0D4F807460CE002
:105B100001F0D0F8C01B0A2807D9606D30436065DA
:105B2000A06D2843A0650120F8BD20680068C0432F
:105B3000C007EDD10020F8BD1700008070B50A4DF8
:105B4000FF22EE1D1346F93605E0047854402A5D25
:105B50005A40335D401C0C46491E89B2002CF4D1DA
:105B60001002184370BD00003AA3000810B50023CE
:105B70001A4603E0845CE3189BB2521C8A42F9D3B4
:105B8000D84380B210BD000010B5034800F0D6FD28
:105B9000024800F0D3FD10BD541600200C16002062
:105BA00030B5446C1C252C400125A540046C656073
:105BB000046863608368102B036803D099600068F1
:105BC000C26030BD9A600068C16030BD10490120DC
:105BD000487202205E31487203203C39487204202A
:105BE0000E3948720A4B0B495A1C0878587149788B
:105BF00099712333187159712033187759771075BB
:105C000051751A461E3210755175107651767047CF
:105C100044110020F000002010B502F011FF2020F8
:105C200002F0A2FF012003F0B7FF002002F09CFF6A
:105C3000044803F055FE044804F0FEF8002004F088
:105C400033F910BDB00000208380000070B505203E
:105C50000121000701F022F800240C4D002800D09B
:105C60002C6002210A4801F019F8002807D10948E0
:105C70002C60008808494000088003F031FB0120B7
:105C800000F044FF022000F041FF70BD0801002039
:105C900000040050D8000020E800002070470000F9
:105CA00010B5084900224A6107494B684C15234347
:105CB0004B604B68082423434B60C009C00102605D
:105CC00010BD00009C160020002002407FB500257A
:105CD0000C460646039500F077FEE009029003A902
:105CE00001960095684600F007FE002804D000F0F9
:105CF0003FFE002004B070BD00F03AFE0120F9E73D
:105D000010B5002302E0C45CCC545B1C9342FAD370
:105D100010BD000010B5214A00219069C30520483C
:105D200004D54169022319434161911593699B058B
:105D300005D54369012423434361630219439369F1
:105D40005B0505D54369082423434361E3011943F7
:105D500093691B0505D5436904242343436163020A
:105D6000194393699B0405D5436910242343436178
:105D70006302194393699B0304D5446920231C43A0
:105D8000446119439369DB0305D5436940242343E8
:105D90004361A0020143916110BD00000020024058
:105DA0009C16002070B5054600F084FF0646184C8E
:105DB0000AE0681C08D0002D04D000F07BFF801B97
:105DC000A84201D9032070BDA069C007F1D1A06924
:105DD000800701D50220A061A069C00511D4A06987
:105DE00080050ED4A06940050BD4A069000508D435
:105DF000A069800405D4A069800302D4A069C0030F
:105E000003D5FFF787FF012070BD002070BD0000A3
:105E100000200240F8B51746002605460C4600F063
:105E2000D3FD09E029460220226800F0AFFD0028DA
:105E300004D1241D2D1D361DBE42F3D300F098FD64
:105E4000BE4201D20020F8BD0120F8BD10B50849BE
:105E500002460020054B497905E044001C5B944252
:105E600003D0401CC0B28842F7D310BD8612002078
:105E70005000002010B5094801F08CF880B2FFF7FF
:105E800031FC074A074BFFF731FB0022064BFFF7B7
:105E900095FBFFF76DFC80B210BD0000C814002018
:105EA000F853E3A59B843E4000408F40F8B5414C39
:105EB000E079002801D0002000E00120E0713D4998
:105EC0003D48CA790275097A41753C490A780276DB
:105ED000497841763A4801783748133001700521F6
:105EE0004172962003F098FF4B20C00003F0AEFFF4
:105EF0003149002213310C2004F078F800210C20E5
:105F000004F086F8022003F0D7FF2E4D00210F2069
:105F100003F0FCFE2842E062F8D0E06A411C3BD06E
:105F2000294E2A4F400439D58122D20100210F2069
:105F300004F031F80021102003F0E8FE41061E486D
:105F4000490E0022633003F017FF1B4D6335687A5A
:105F5000052820D102221949681DFFF733F90028CE
:105F600019D1A87A607113480422691C4030FFF7E8
:105F700005F9206C00F02EF8608360792946420014
:105F80000B3108467330FFF7F9F8608B31884843CE
:105F9000388002202070F8BD02F0C2F80C48018859
:105FA000608B0546FFF7A4F83088414339806D1EA9
:105FB0006583F8BD50000020A5110020F0000020EE
:105FC000C700002000D02724D2000020D0000020ED
:105FD000D400002010B504460E4800F0DBFF0E4947
:105FE000C006C00E098805E02246C240D2070FD085
:105FF000401CC0B28842F7D3012005E02246C240CF
:10600000D20705D0401CC0B28842F7D3491EC8B29F
:1060100010BD0000C8140020D400002010B50848AE
:1060200000F038FB0A21064800F0D4FA044800F0DA
:10603000ABF9800503D5024800F0A8F980B210BD85
:106040006C140020F8B5384C4B216088C900054617
:10605000FFF74EF86D1C6580002960D101F0F4FE59
:106060001E2000F03BFCFFF7D9FFE08001F0E2FECC
:106070002E48008BA080E088FFF718FB0546A0881B
:10608000FFF714FB2A4F3946FFF702F92946FFF7BD
:106090003CF9FFF78BFB274A274BFFF775F9FFF712
:1060A00099FB002605462061B84237DB6078234F14
:1060B00000280ED066702846FFF778FB00223B468A
:1060C000FFF706FA00221E4BFFF710FAFFF782FBDC
:1060D000E0602846FFF76AFB00223B46FFF7F8F92D
:1060E000184A194BFFF702FA05460F46E068FFF71A
:1060F0005DFB144A154B5242FFF7F8F92A463B461E
:10610000FFF742F9FFF766FB1149E060884201DDC5
:10611000E16004E0FF21C905C84200D3E660E06801
:10612000FFF7EEFAC0B2F8BD240000206000F81FAF
:1061300000004040A4703D0AD7A3C03F00000840C3
:1061400000E064403333333333B33040CCCCEC3FE6
:106150000000C842F8B5054604464035287C0026B4
:10616000012808D001202874206881688907890FD8
:1061700001290ED101E00220F8BD0168C90708D04D
:10618000606D202108436065012600202874304698
:10619000F8BD616DFF220132914302221143616516
:1061A000C1688907890F0091C16889088900C160A9
:1061B0002068816892071143816000F07BFD0746EB
:1061C0000EE000F077FDC01B0A2809D9606D02219E
:1061D0008843102108436065002028740120F8BD21
:1061E000206880680028ECDB2068C168009A1143B1
:1061F000C160606D80088000401C6065C5E70000DC
:106200000248016A82159143016270470000014013
:1062100070B50A4D286AA9150843286200F04AFDA6
:10622000044606E000F046FD001B032801D90120CA
:1062300070BD286A4000F5D5002070BD0000014007
:10624000F8B506460D464036317C01290DD00121B6
:10625000317401688A68520709D5416D20221143C3
:106260004165002030740120F8BD0220F8BD174BB5
:106270006A68D80547109A42154C8A6A2B6812D072
:106280005B035B0B1A438A622968490305D5A16841
:106290000143A1600A20FFF7DDFB2868800312D5C7
:1062A000A06838430EE05B035B0B9A438A6229685F
:1062B000490302D5A1688143A1602868800302D503
:1062C000A068B843A06000203074F8BD0110000041
:1062D0000027014070B5040043D0606D02210843DF
:1062E00060652046FFF78CFB0026054600283AD063
:1062F000012D32D0206841681F4A11404160216859
:10630000D0430860206881680122120791438160B0
:106310002068C168194A1140C16020680169184AA3
:106320001140016120684169C908C90041612068C4
:10633000016A144A1140016220688030416BC9092A
:10634000C901416320688030416BC909C9014163BB
:10635000204600F003F9A665666540342674284699
:1063600070BD012070BD2046FFF786FB0546012861
:10637000F3D001206065BDE760F7FFFF00023E83B8
:1063800002FCFF3F00F000F0406D70470068006CB9
:106390007047000070B5040006D0606D26460025E9
:1063A0004036002802D006E0012070BDA565357496
:1063B000204600F0E7F8606DC00603D421688868C5
:1063C000400705D5606D1021084360653574EBE723
:1063D000606DFF220132904302221043606588689D
:1063E0008207920F5B48012A02D10A68D2072BD19B
:1063F000032362689B079A4205D05B429A4202D00F
:106400005B009A4209D10A69920092080A612168E8
:106410000A6963681A430A610CE00A6992009208EB
:106420000A6181680F2292049143816081686268E9
:10643000114381602168CA6818239A43CA602168A1
:10644000CA68A3681A43CA60816801225206914350
:1064500081608168A28E5206114381602068816844
:10646000C90004D4816801221207114381602068A9
:10647000C168394A1140C1602069E168022825D00D
:1064800000200143204620300278037B52035B004A
:106490001A431143226B1143A26992031143E2692B
:1064A000D20311432268D3681943D160616A0A4656
:1064B000FF3AC23A05D0A26A11432268D368194351
:1064C000D16042780121012A02D00BE00420D8E7F4
:1064D0000078002823D0606D202210436065A06DF5
:1064E0000843A065E06B012820681FD00169C90737
:1064F00003D0016949084900016120684169C90860
:10650000C900416120684169A26B11434161A565E1
:10651000606D80088000401C6065002070BD2068B0
:10652000C26801231B041A43C260DBE70269FF2330
:106530009B009A43026120680269236CA66C1A438F
:10654000636C33431A430261206802690A430261A3
:10655000D3E70000002701401902FEFF10B50068D4
:106560000649884209D10648416B4215914341636F
:1065700005200221000700F055FA10BD002401405B
:106580000010024010B586B0044614216846FEF79C
:106590000EFE0E492068884216D10D48416B421507
:1065A00011434163C16A01221143C162C06A694655
:1065B00010400590022000900320019000200290DE
:1065C0000520000700F0AEFA06B010BD002401401F
:1065D00000100240F8B504464069254640350E4695
:1065E00008280BD02068C068C00709D0606D202142
:1065F00008436065002028740120F8BD082700E0EA
:106600000C2700F057FB009011E0701C0FD0002EFB
:1066100005D000F04FFB0099401AB04207D9606DD9
:10662000042108436065002028740320F8BD206819
:1066300000683842E9D0606D012149020843606575
:106640002068C16809058A0F0C21002A1BD120226D
:10665000125D002A17D10268120714D58268530709
:106660000122002B08DB43688B434360606D1302FB
:1066700098431043606506E0606D20231843606511
:10668000A06D1043A065A069002801D120680160B9
:106690000020F8BD70B504462168002089684907CC
:1066A00021D425464035297C01291CD0012129749B
:1066B000E169012904D02046FFF70EFA002811D124
:1066C000616D0A4A1140FF220132114361650021C8
:1066D000A165297422681C21116021688A6804233D
:1066E0001A438A6070BD022070BD0000FEF1FFFFFA
:1066F00070B50024014620314A79022A03D00421D2
:10670000C163012418E0026813680E25AB431360CF
:10671000026813685B085B001360436C1C22134023
:10672000012215469D40036C5D604A7100220A718A
:10673000816B002900D08847204670BDF0B4016C01
:106740000D6801680C68466C1C2304221E40174625
:10675000B7402F420ED067070CD50C68A40602D4B0
:106760000C6894430C60416C19408A40016C4A608B
:10677000016B1AE00227B74002462F402032002F5B
:1067800017D0A70715D50C68A40605D40C680A25F0
:10679000AC430C6001215171446C02211C40036C1C
:1067A000A140596000211171C16A002918D0F0BCC4
:1067B00008470827B7402F4212D0240710D50C688D
:1067C0000E25AC430C60446C01211C400B46A340D9
:1067D000046C6360C163517100211171416BE4E786
:1067E000F0BC704770B504003CD01F4825681421E8
:1067F0002818FEF77DFC800060641C48206402219C
:10680000204620300246417129681948E36801405A
:10681000A06866691843236933431843A369184382
:10682000E3691843236A1843084328600121A068DC
:106830008903884210D00D488030836A656C1C2122
:106840000D400F26AE40B3438362656C63680D4014
:10685000816AAB400B4383620020E06301215171E8
:10686000107170BD012070BDF8FFFDBF0000024037
:106870000F80FFFFF8B504468C46203001790025D3
:10688000012909D00126067141790027012905D087
:10689000077102252846F8BD0220F8BD022141718A
:1068A000E7632068016849084900016061462046A5
:1068B000FFF776F9206B00282068016801D00E22CE
:1068C00005E0042291430160206801680A22114317
:1068D00001602068016831430160DBE770B5044660
:1068E00000F0E8F90546601C00D0641C00F0E2F9F5
:1068F000401BA042FAD370BDF8B51A4E0546307C55
:106900000F46012807D0012030741748FFF74AFAD4
:10691000010002D021E00220F8BD0020C043386011
:106920006C6814E02046FFF7BBF90F48FFF73AFA0E
:1069300001460E48426808239A4342604268431564
:106940009A434260002901D03C6006E08034A86888
:106950006A68C0018018A042E4D80020307408465C
:10696000F8BD00009C16002050C30000002002402B
:1069700005484168022211434160416801221143E8
:10698000416000207047000000200240F8B50C4C28
:106990001646207C0F46012808D0012020740948A3
:1069A000FFF700FA0025002802D006E00220F8BD1B
:1069B00065613E600348FFF7F5F92574F8BD0000F6
:1069C0009C16002050C3000011484168C9070BD035
:1069D000EFF3108172B60F4AC2600F4AC26081F3B2
:1069E00010884168C9070ED1416889070DD5EFF3BA
:1069F000108172B6094A0261094A026181F3108866
:106A00004068800701D501207047002070470000D2
:106A100000200240EFCDAB8905040302BFAE9D8C80
:106A200016151413F0B500235DE001249C402246A6
:106A30000A4057D006685F000325BD402E43AC4690
:106A40000660DD08AD002D182E6AAE465D07EF0E1C
:106A50000F25BD40AE4375462E6286686546AE433F
:106A600086604568A5434560C4686546AC43C4601C
:106A70009D081F4CAD002D19AF689C07260F0F24F1
:106A8000B440A4463C4005273F07B84201D1002747
:106A900014E0184FB84201D101270FE0164FB84259
:106AA00001D102270AE0154FB84201D1032705E0C2
:106AB000134FB84201D1052700E00627B740A7428F
:106AC00010D1AE686446A643AE600E4C256895436F
:106AD0002560656895436560A5689543A560E56890
:106AE0009543E5605B1C0A46DA409ED1F0BD00008C
:106AF000000001400004005000080050000C00504D
:106B0000001C0050000401407047000010B504490B
:106B10004A69024202D04861FFF7F6FF10BD00004B
:106B200000040140F8B500230124A2E027469F405D
:106B30003A4070D04D68022D01D0122D14D1DD08DD
:106B4000AD002D1800952D6A5E07AC46F50E0F2698
:106B5000AE46AE406546B543AC460E697546AE409E
:106B600065462E43009D2E624D68012D05D0022DF5
:106B700003D0112D01D0122D16D185680326AC4605
:106B80005D00AE46AE406546B543AC46CE68754640
:106B9000AE4065462E43866046680D79BE43ED06DD
:106BA000ED0F9D403543456006685F000325BD40FD
:106BB000AE46AE430D79B446AE07B60FBE4065464D
:106BC0002E430660C6687546AE438D68BD403543AA
:106BD000C5604D68ED004BD5294D6E6B26436E6345
:106BE0009E08284DB6007519AC46AD689E07360F55
:106BF0000F27B740BD4305273F07B84201D1002703
:106C000015E0214FB84201D1012710E01F4FB842D3
:106C100002D102270BE02BE01D4FB84201D1032720
:106C200005E01C4FB84201D1052700E00627B74018
:106C30002F436546AF60184D2E684F689643FF039B
:106C400000D516432E606E684F689643BF0300D58B
:106C500016436E60AE684F689643FF0200D5164338
:106C6000AE60EE684F689643BF0200D51643EE60F3
:106C70005B1C0A681546DD4000D057E7F8BD0000F0
:106C800000100240000001400004005000080050C5
:106C9000000C0050001C0050000401400069084036
:106CA00000D001207047002A01D0816170478162C5
:106CB0007047000001480068704700000C01002088
:106CC00002480168491C0160704700000C01002067
:106CD00010B5084800240168402211430160204695
:106CE00000F00AF8002801D0012401E000F07EF94C
:106CF000204610BD0020024070B5054609487D21A0
:106D00000024C9000068FEF7F3F900F0CFFD002869
:106D100001D0012404E000222946501E00F07CF935
:106D2000204670BD1001002070477047F8B5294C0F
:106D3000A078401CA07001202071608C401C6084F1
:106D4000A08901F0E5FE244DE888FEF7AFFC234F53
:106D50003946FEF7DAFA224E00903168FEF73FFA24
:106D600030600120216BC005814203DB0098FEF7F3
:106D70008BFA20631B4E02213046FFF78FFF00285D
:106D800002D00020E063F8BDE888FEF78FFC3946AA
:106D9000FEF7BBFAE16BFEF722FA1349E063884283
:106DA000F1DB207A002813D000210B48403081808D
:106DB00003F044FA0121002289023046FFF773FFF5
:106DC0007D200001FFF78AFD09490848C860F8BD29
:106DD0000121EAE7C4000020440D002000007A44AD
:106DE00008010020000400500000A0400400FA0543
:106DF00000ED00E070477047704710B5044600682A
:106E00000168C943C90708D18168C943C90704D1CA
:106E1000012141602046FFF789FF20680168C943CE
:106E2000890708D48168C943890704D402214160D5
:106E30002046FFF779FF20680168C943490708D455
:106E40008168C943490704D404214160204600F009
:106E5000CBF820680168C943090708D48168C94391
:106E6000090704D4082141602046FFF7C3FF2068CA
:106E70000168C943C90608D48168C943C90604D456
:106E8000102141602046FFF750FF20680168C94388
:106E9000890608D48168C943890604D42021416049
:106EA0002046FFF7A9FF20680168C943490608D4B6
:106EB0008168C943490604D4402141602046FFF758
:106EC0009AFF10BDF8B5040005D025462035A87BF3
:106ED000002802D006E00120F8BD0020687320469B
:106EE00000F040F80220A8732068C26884466368F6
:106EF000012B04D00120A16AC005814201D11E20CE
:106F0000824315486169814201D014480240144807
:106F1000A668024018463043676A266A3E433043FB
:106F2000A66A30431043012B03D00122D2059642BA
:106F300003D12369E2681A431043074A914205D0FE
:106F4000A2691143E2690243084610436146C860E2
:106F50000120A8730020F8BDFFFF00003F1FFFFFC6
:106F6000F8F119FF10B50068084988420CD10848AB
:106F7000816BC20411438163002201210D2000F0C6
:106F80004BF80D2000F03EF810BD0000007C0040E2
:106F9000001002400068C0697047000070B502240C
:106FA000034620339C730F4C2568E6043543256067
:106FB0000468E568B6123543E5600568AE680124EB
:106FC0002643AE6005682E6926432E610568A961D7
:106FD00001684A61006801690422114301619C73E0
:106FE000002070BD00040140704700000448416B60
:106FF000012211434163816B020411438163704795
:1070000000100240C106C90E0120884001490860F5
:107010007047000000E100E010B501F05FF810BD1E
:1070200002480168821511430160704700700040FA
:10703000F8B504460078544D800672D5524E0027AC
:10704000403EB06BC00004D4B06BA9050843B063E8
:1070500001274E480168C90511D401688215114302
:107060000160FFF727FE009005E0FFF723FE00997F
:10707000401A642837D845480068C005F5D53268FD
:107080000321090560680A400140914208D081034C
:10709000890F032904D13168890301D50120F8BD86
:1070A0002A69032109040A4022D0084090421FD0D7
:1070B000207880061CD528692A6988430121C904E3
:1070C0000A432A612A698A432A612861C0050FD5CB
:1070D000FFF7F0FD009008E0FFF7ECFD0099411A82
:1070E0002B48814201D90320F8BD28698005F3D5DA
:1070F00061688803800F032805D132680005824348
:1071000001400A4332602869032261681204114079
:1071100008432861002F04D0B16B01200007814390
:10712000B1632078C00705D0E868A16880088000B6
:107130000843E8602078800705D5E8680C2188437B
:10714000E1680843E8602078400706D5E868032135
:107150008902884321690843E8602078000706D542
:10716000E86803210903884361690843E8602078DF
:10717000000606D5E868032189048843A16908430D
:10718000E8600020F8BD00004010024000700040A0
:1071900088130000F8B50E4605007DD053480068FE
:1071A000C007C00FB0420AD25048016849084900E0
:1071B000314301600068C007C00FB04271D1287828
:1071C0004B4C800705D5E068F0218843A968084347
:1071D000E0602878C00752D06868022817D00328DA
:1071E00018D02168012818D08905002959DAE168EA
:1071F000890889000143E160FFF75CFD6968074683
:10720000022912D003291CD0012926D033E021689D
:107210008903EAE721688901E7E74907E5E7FFF71E
:1072200049FDC11B3348814223D8E0680007800F25
:107230000228F4D123E0FFF73DFDC11B2D48814218
:1072400017D8E0680007800F0328F4D117E0FFF794
:1072500031FDC11B274881420BD8E0680007800F31
:107260000128F4D10BE0FFF725FDC11B2148814225
:1072700001D90320F8BDE0680007800FF3D11B4857
:107280000168C907C90FB1420DD901684908490011
:1072900031430160006800E003E0C007C00FB04266
:1072A00001D00120F8BD2878400706D5E068072105
:1072B00009028843E9680843E0602878000707D599
:1072C000E0680721C90288432969C9000843E060D2
:1072D00000F036F8E168084A0906090F515CC84019
:1072E000064908600020FFF707FDF8BD00200240B6
:1072F00000100240881300003AA500081001002089
:10730000044805490068C968044A4905490F515CA9
:10731000C8407047100100200010024053A500082B
:10732000044805490068C968044A8904490F515C4A
:10733000C8407047100100200010024053A500080B
:1073400010B5184AD1680C20084004280BD0082832
:1073500010D00C2810D050680004410F0120C00349
:10736000491C884010BD1068C00601D50E4810BDEC
:107370000E4810BD0E4810BD88020E4B000F185C61
:107380000902D368890F491CDB0301D5084A05E0CF
:107390001268D20601D5044A00E0044A5043FDF7C2
:1073A000A7FE10BD0010024000093D000024F400BB
:1073B00000127A004AA50008FEB505007ED0FE4CFA
:1073C000E7680C20E66807400120000406402878A2
:1073D000C00747D0082F05D00C2F0AD10120000488
:1073E000864206D1206880033CD568680028E5D035
:1073F00038E0012069680004814203D1216801431B
:10740000216011E0052301221B04920499422168A6
:1074100002D111432160F1E78143216021680140DD
:107420000091206890432060686800280DD0FFF725
:1074300041FC009005E0FFF73DFC0099401A6428EC
:107440007AD820688003F6D50CE0FFF733FC009073
:1074500005E0FFF72FFC0099401A6428F0D8206857
:107460008003F6D42878800755D50923E868042FCF
:107470000DD00C2F01D1002E09D000283BD021685F
:10748000994301432160FFF715FC064627E0216878
:10749000490701D5002891D061681F22120291434B
:1074A0002A691202114361602168994301432160F6
:1074B000FFF746FFE16809060A0F00E079E1BF49DE
:1074C000895CC840BE4908600020FFF715FC002811
:1074D00072D120E0FFF7EEFB801B0228B0D82068B5
:1074E0004007F7D560681F2109028843296909020E
:1074F000084360600FE02068400840002060FFF70C
:10750000D9FB064604E0FFF7D5FB801B022897D87D
:1075100020684007F7D42878C0065FD5002F0CD02C
:10752000A869002849D02068FF2101310843206064
:10753000FFF7C0FB06462DE0C0E02068800502D5BD
:10754000A8690028A7D06068072149038843296AF1
:10755000084360606068297F0002000A090608434A
:107560006060286A410B0120C003491C8840E16823
:1075700009060A0F9149895CC840914908600020BA
:10758000FFF7BAFB002817D128E0FFF793FB801B19
:107590000228A3D820688005F7D560680721490331
:1075A0008843296A084360606068297F0002000AF6
:1075B00009060843606011E0E1E02168FF20013026
:1075C00081432160FFF776FB064604E0FFF772FB7C
:1075D000801B022872D820688005F7D42878794E5D
:1075E000000724D568690028306910D001210843BC
:1075F0003061FFF75FFB009005E0FFF75BFB009950
:10760000401A02285AD830698007F6D50FE04008A2
:1076100040003061FFF74EFB009005E0FFF74AFBAA
:107620000099401A022849D830698007F6D4287892
:10763000400765D500200290A06BC00006D4A06B67
:10764000012109070843A063012002905E480168F8
:10765000C90511D40168821511430160FFF72AFBA7
:10766000009005E0FFF726FB0099401A642825D812
:1076700055480068C005F5D5FF20AA680130824250
:1076800003D131690143316111E001218902002AEE
:1076900007D005231B029A4203D132690A433261A3
:1076A000EFE7326982433261306988433061A8680C
:1076B00000280FD0FFF7FEFA009007E05EE0FFF72A
:1076C000F9FA0099411A4148814257D8306980053A
:1076D000F5D50DE0FFF7EEFA009006E0FFF7EAFAC5
:1076E0000099411A3948814248D830698005F5D45B
:1076F0000298002804D0A06B012109078843A063E9
:10770000686A002864D00C2F3ED001263606022875
:10771000206805D0B0432060FFF7CCFA05462FE083
:10772000B0432060FFF7C6FA074604E0FFF7C2FA4D
:10773000C01B022822D820688001F7D4E96AA86A11
:10774000E2680843296BFD231B049A431143084355
:10775000E060206830432060FFF7ACFA054604E0A3
:10776000FFF7A8FA401B022808D820688001F7D547
:107770002EE0FFF79FFA401B022801D90320FEBD2F
:1077800020688001F5D423E00128F8D0E0680121C9
:107790000904AA6A014091420BD10F218904EA6AC7
:1077A0000140914205D1032189050840296B884297
:1077B0000ED00120FEBD0000001002403AA50008D6
:1077C00010010020401002400070004088130000AB
:1077D0000020EFE770B5040007D0002625464035AD
:1077E000A662687C002802D005E0012070BD2E74DE
:1077F000204600F02FF802206874206801684022BB
:1078000091430160A168606822690843E1681143FF
:107810000843616901220843A169520211400843EB
:10782000E1690843216A0843A16A084321680860A6
:10783000A0690421000C0840616A0843216848607F
:107840002068C16992009143C16166650120687436
:10785000002070BD10B586B0044614216846FDF7BF
:10786000A6FC10492068884219D10F48416B821448
:1078700011434163C16A01221143C162C06A002100
:1078800010400590E020009002200190032003901A
:1078900002910491052069460007FFF743F906B0FD
:1078A00010BD00000030014000100240094910B531
:1078B000401E884201D9012010BD074C60610321A0
:1078C000081F00F00BFC0020A061072020610020B1
:1078D00010BD0000FFFFFF0000E000E070477047B0
:1078E000F8B502680446D0691168936805072D0F42
:1078F0005BD0DD07ED0FFF2621360E402E4367D00B
:10790000C60706D0CE0504D501261662E26F3243C3
:10791000E267870702220426002F06DADF0704D079
:1079200027683A62E76F3743E767470706D5DB0703
:1079300004D023681E62E36F1343E367020709D58F
:1079400020220A402A4305D0236808221A62E36FE6
:107950001343E367E26F002A2FD0800606D588061E
:1079600004D5216E002901D020468847E06F2168A8
:107970008968490601D4000724D5204601F00EFB92
:1079800020688168490619D5816840229143816049
:10799000E06E002812D020498163E06EFEF7A8FE59
:1079A00000280AD0E06E816B06E0850610D58D06B2
:1079B0000ED5216E1CE020468847F8BD2046FFF713
:1079C0008EFFF8BD2046FFF78AFF0020E067F8BD74
:1079D000C50208D55B0206D50120000510622046CD
:1079E000FFF77CFFF8BD030605D50B0603D5616ED6
:1079F0000029E0D1F8BD4006FCD54806FAD5136849
:107A0000204640218B43136020216167002161667D
:107A100000F069F9F8BD0000F98E000810B5040007
:107A200003D0606F002802D007E0012010BD0021C4
:107A300070200155204600F027F824206067206858
:107A40000168490849000160204601F0F1FA012867
:107A5000ECD0606A002802D0204601F031F920689D
:107A600041680922D20291434160206881682A223C
:107A70009143816020680168012211430160204622
:107A800001F084F910BD0000F0B587B0064614215E
:107A90006846FDF78CFB2C493068884251D12B4851
:107AA000416B0122920311434163C16A01221143D8
:107AB000C162C06A0025104005900320400200907A
:107AC0000220032701A9A1C10420049005206946D2
:107AD0000007FFF727F81F4C1D48A560E56081C42B
:107AE0008027E560A7602020256160610002A06119
:107AF0001848083CFEF776FE002801D0FEF7CEF8C5
:107B0000F466A662144C1248214614382060032003
:107B1000606010200831A1C16561A561E561204662
:107B20002562FEF75FFE002801D0FEF7B7F8B466C5
:107B3000002201211B20A662FFF76EFA1B20FFF72F
:107B400061FA07B0F0BD00000038014000100240AB
:107B5000300002400C16002054160020F8B50446F0
:107B6000806F20284DD100290BD0002A09D0012395
:107B7000A0681B03984206D12069002803D1C807DA
:107B800001D00120F8BD25466035287C012838D079
:107B9000012028745820616502530026E6672220E0
:107BA000A067E06E002819D01749C162E16E17483E
:107BB0000863E16E16484863E06E13468663676D9E
:107BC00021683A462431E06EFEF754FE002805D0C5
:107BD0001020E0672E7420206067D2E72E742068A2
:107BE0000168FF220132114301602068816801228F
:107BF0001143816020688168402211438160002028
:107C0000F8BD0220F8BD0000558F0008938F0008D2
:107C10000D8F000870477047FFB50446406F83B072
:107C200017460D4620285CD1002D0AD0002F08D021
:107C3000A168C001814207D12069002804D1E8076A
:107C400002D0012007B0F0BD204660300290007CD9
:107C5000012846D00298012101740020E06721200C
:107C60006067FFF727F82646403601903782778213
:107C70000120A1680003814202D12069002802D0BE
:107C80002F46002511E000270FE00022802120462A
:107C900001F0E2FA002815D1002F15D021683878BC
:107CA00088627F1C708A401E7082708A019B002847
:107CB00006980090E9D100224021204601F0CCFA3C
:107CC000002808D00320BDE728882168C005C00D22
:107CD0008862AD1CE6E720206067029900200874E6
:107CE000B0E70220AEE7704701490248C160FDE7F6
:107CF0000400FA0500ED00E0F8B53C480068C069F2
:107D00003B4E3C4F800700D5FE600121C9023A4836
:107D1000FEF7C4FF394C0025002827D001F066F893
:107D200001F09EF836480560E079002803D1012073
:107D3000E07101F0D5FA2078632806D900220821E5
:107D40002D48FEF7B0FF012205E0012208212A4854
:107D5000FEF7A9FF002201210520C9030007FEF755
:107D6000A2FF284CA08C012803D01CE0E571002262
:107D7000ECE725486946088072B680212348FDF764
:107D8000A5FF002804D0022269462048FEF742F8E9
:107D900062B61FA001F040FBA58402F04FFA6420F8
:107DA00001F050FDFE60608C012809D11548658402
:107DB0004038058002F042FA642001F043FDFE6085
:107DC000208C012806D1258402F038FA642001F0C5
:107DD00039FDFE600B48124A40380188914202D1B9
:107DE000C088002800D1FE60F8BD00008C1500207E
:107DF0000400FA0500ED00E000040050C40000207B
:107E000008010020840D0020AAAA0000384A0008BA
:107E1000BDF8C8EBC9FDBCB6C4A3CABD0D0A0000BD
:107E2000AA55000010B50248FEF7E7FF10BD00009C
:107E3000C814002010B50348FEF74CFAFEF7E0F92D
:107E400010BD00006C1400201CB5002118480091E2
:107E5000164A01910260C1631205426081600722E7
:107E60008263012202610246C16020321170FF2349
:107E70005170C233436281621173016381610422D4
:107E800041634261C161FEF785FA0A480090012012
:107E90000003019069460648FEF7D2F9FEF7B8F9EB
:107EA00000210348FEF756F91CBD000000240140E4
:107EB0006C1400200000024408B50848016B012240
:107EC00011430163006B01211040009000220A2041
:107ED000FFF7A2F80A20FFF795F808BD001002404E
:107EE000F0B587B014216846FDF761F94748C26ACA
:107EF00004210A43C262C26A0A400592C16A80260E
:107F00003143C162C16A31400591C16A01242143F4
:107F1000C162C16A21400591C16A02252943C1623B
:107F2000C06A22462840059005201C210007FEF764
:107F3000BAFE012236493748FEF7B5FE002236491F
:107F40003448FEF7B0FE9121052000220902000707
:107F5000FEF7A9FE314801900027052069460297E7
:107F600000940007FEF7DEFD0C2000901120019028
:107F7000032003900520029769460007FEF7D2FD13
:107F800010206A46039591C2052069460007FEF756
:107F9000C9FD1120019002976946039700941D487E
:107FA000FEF7C0FD1E4801906946009502941948ED
:107FB000FEF7B8FDE002009069460197029515486A
:107FC000FEF7B0FD1748694691C16946114803970D
:107FD000FEF7A8FD91200002694691C1052069467F
:107FE00000070397FEF79EFD69460A480197009631
:107FF0000294FEF797FD002201210520FFF70CF8FF
:108000000520FEF7FFFF07B0F0BD000000100240A2
:1080100001020000000400500830000000001110B0
:10802000000021100832000010B50F4C0D482060F0
:10803000FF20053060600020A060E060206160618A
:10804000E0610121206249026062A161A062072013
:10805000E0622046FFF7BEFB206801684022114322
:10806000016010BD00300140F814002000B585B05B
:1080700014216846FDF79BF8164815490160E12177
:108080004902416000218160C160016181610C226F
:10809000C1614261016230214162012109038163B2
:1080A0004900C163FFF7BAFC012080020090022062
:1080B00001900120029003200390042004900520E9
:1080C00069460007FEF72EFD01F004F905B000BD7A
:1080D000003801408C150020704700008307FF2204
:1080E000DB0E9A408907090E994000280BDA000739
:1080F000000F0838830808489B001818C369934389
:108100000B43C3617047830804489B001B18186821
:10811000904308431860704700ED00E000E400E081
:10812000BFF34F8F04490348C860BFF34F8F00BFB0
:10813000FDE700000400FA0500ED00E0F0B58FB0A7
:1081400000200C90962001F067FEFE4801F07EFEB4
:10815000FD4F00247C70B87B0C2801D30B20B87332
:108160000122052051020007FEF79DFDB87B7873C0
:108170007871F648BC70F64D00782870F5480221F9
:1081800000782871F448FEF789FD00285ED00020B1
:10819000B979EF4D49000843E871B86AE870401CAE
:1081A000B86278792946A8724200CE310846C338B1
:1081B000FCF7E4FF06206872284613380490397FE4
:1081C0000175797F417578790022400029460D308C
:1081D00001F00CFF7879002140000D3001F018FF0C
:1081E000022001F069FEEC713C74BC72012038730E
:1081F000FC72DA48FEF7CEFE38840546BC7078790A
:10820000FDF770FAD64AD74BFDF770F90022D64B2E
:10821000FDF7BAF8FDF7ACFA0006C00C401980B2C1
:108220000121C9037884884201D3401A7884CF4859
:108230007863F878401CF870C848FEF7ABFEF88306
:10824000C3480A300B9044300A901EE201209FE799
:10825000C248FEF79FFEF883C54DC64E3EE0B87A91
:10826000002830D001F099FD069988422BD9059954
:10827000884228D201F068FC3C730C98002819D081
:10828000B348202141726622BB490B98FCF776FF68
:108290006621B948FDF752FC69460880AC490022C6
:1082A0006C3188806C39742001F0A0FE00217420AC
:1082B00001F0AEFE099801F0A8FD012001F0FCFDDF
:1082C0003872BC7211E0A548FEF764FE80B2F883F4
:1082D000798C884202D38919884206D300210F2065
:1082E00001F014FD2842F862B9D0F86A411C1ED092
:1082F00040047DD58122D20100210F2001F04BFEE8
:108300000021102001F002FD41069148490E002293
:10831000503001F031FD002001F098FD002001F007
:108320004AFD8B4D5035687A07288ED101E0FFF762
:10833000F7FE02229149681DFCF744FF002884D112
:10834000834850300178814800788142EDD1002681
:10835000354607A801F027FD042007AA310E2D029B
:108360000D433102165C0E43401EF7D5BE64FD641A
:1083700000263546104601F008FD042007A9320EFC
:108380002D02154332020E5C1643401EF7D53E65A2
:108390007D65B9786E4A491CB9704D3216796946C7
:1083A0000E7052794A706A4902925031C97C0D09A7
:1083B000BD740AD066493D74072266317048FCF7E7
:1083C000DDFE022D01D101200C90787B3D46002876
:1083D0000BD10120287169460A885D49CE310A8097
:1083E000687104980675029941755948CE3000E0CD
:1083F00040E1018868460088039081427ED10A9856
:10840000604E008A308052484C30808A288353481E
:10841000FEF7C0FDE883288B5B49FF30C33080B294
:10842000288388420BD94942401828833188564A0C
:10843000491C89B20B323180914200D334805048BC
:1084400003210C3801700A983F4A81891186C0893E
:108450004B4B50869C3B2A6B1A601A46B03AD27C32
:108460001207120F032A00D06A74EC700122AA725C
:10847000354A9186D0866879FF2191314843424937
:108480002A6D593940180004C1176B6D8018594185
:108490000906000A08433D49099040180690192131
:1084A0000998890240180590099840084000010E7B
:1084B0000002E965A865EB6CAA6C0B9801F0CEFD93
:1084C00023486B6D16302A6D01F0C8FD2048EB6D16
:1084D0001230AA6D01F0C2FD1D48082141721B49EE
:1084E0000022097801706879194980001C3001F078
:1084F0007DFD6879002180001C3000E078E001F00B
:1085000087FD0120E87212490F48042251314030A2
:10851000FCF734FE36887D20C000298B704340185C
:10852000A8630D901A480078E87302901248C0883A
:10853000FDF7BCF801903046FDF7B8F80199FCF75B
:10854000E4FE27E01027000050000020C7000020B4
:10855000B8110020C400002000040050C8140020FE
:10856000666666666666E63F00001040A08601000B
:1085700000D02724983A0000440D0020F00000208D
:108580005413002004010020E703000000AEFCFFAC
:10859000E60000207F21C905FCF721FEFDF7B0F8B9
:1085A00081B2B94801800298401E814201D1012068
:1085B000E872AE841420285EFDF780F807910290DF
:1085C000E88BFDF78FF8B14AB14BFCF78FFF0646F9
:1085D00003910D98FDF772F83246039BFCF778FF84
:1085E000079B029AFCF7D0FEFDF79EF8E8634CE08B
:1085F000FDF72CFC697B88420CD301212971697934
:10860000A44A491C697143000399D15204990E751B
:10861000029A4A759F4A0321C23211540A999E4A0E
:108620008B891386C989518681009A482A6B32301A
:108630004250B038C07C6B7C0207120F9A4202D9BC
:10864000032A00D0687493486B6DCE380818163032
:108650002A6D01F003FD68798E4980000022CE3931
:108660001C3001F0C3FC6879002180001C3001F04F
:10867000CFFC0AE02A4600210F2001F08CFC387B59
:10868000002802D0002001F096FBF98B788C814203
:1086900000D2DDE5814A80188142FAD880480088FE
:1086A00081004018F978884200D27C747D4A00210C
:1086B0000F2001F070FCB87878710020B8737A7BD5
:1086C0003B790146D31821E0724CC234225C002A67
:1086D0001AD0BD7B8C006D1CBD736E4DA4469235C7
:1086E0002A516C4C45004E00655B1834A55385003B
:1086F0001A34684E6559644662363551491C344611
:108700006034521EC9B22254401CC0B28342DBD82E
:10871000F878012810D95F48C230007800280BD0C3
:108720006148FEF737FC6149C9880901FCF7E0FCA4
:108730005F4802888918018057490022887B487366
:108740000490401E33E000212DE0524C8B00623437
:108750001E19B446E5587668B54222DD06954D4DA2
:108760004C0018352F5B7A35BE469700ED590595BC
:10877000484D77466235EE504A3D6519454E0B959A
:108780006D881836355334467A341E19414D746855
:108790009235EC506346069D5D600B9D6F80059D94
:1087A0007560491CC9B28142CFDB521CD2B28242F1
:1087B000C9DB394C00206072049A2AE03549450033
:1087C00018314B5B18394B53324B324E81006233B8
:1087D0005B5832367350374EB34218D02D4B92331C
:1087E0005B58032B13D1637A06271E467E43294F1D
:1087F0001A3FF6191A37ED192D88B5803D463235E6
:1088000049190D88F580498831815B1C6372401CD1
:10881000C0B29042D2D31F4A002026493232830090
:10882000401CC0B2D1500C28F9D31E4A002180321E
:108830000F2001F0B0FB207C012823D11548052131
:10884000CE30FDF77BF96946124C8880CE34022287
:10885000611D01A8FCF7B6FC002813D123786078CD
:10886000A278022B0ED101280CD0C8280AD20F4BB7
:10887000E11C1818FCF782FC01F0E0FC642000F019
:10888000E1FF54E50FB0F0BDE6000020F853E3A58A
:108890009B843E408612002050000020983A000041
:1088A000D800002000D02724C8140020440D002048
:1088B000CE000020FFFF010070470000FEB54449D4
:1088C0004248086001F05AFC424800F0E1F8424C8E
:1088D00060834048801C00F0DBF8A0833D48001D09
:1088E00000F0D6F8E083FF203C4D2C30688028460D
:1088F0004030017921720291E88E3949C0B2087086
:108900000190E88F6071A88FA071A87AE070A888A4
:108910000090E0622889FCF7E5FE324A324BFCF712
:10892000E5FD00F02BFF0022304BFCF72DFDFCF79E
:108930001FFF86B2E681EF8831463846FCF7D8FB48
:10894000208201460098FCF7D3FB71438EB27D2054
:10895000C000A6817043FCF7C5FE254A254BFCF7F5
:108960002DFEFCF705FF60827D20E6823946C000BF
:10897000FCF7BEFBA0822084688F60720299012000
:10898000002902D160710A216172002F01D1642196
:10899000E980019A1249432A01D943220A7060846E
:1089A000FDF768FA2083628A13491448FEF7F6FA45
:1089B00013A0E16A00F030FDE98815A000F02CFD5D
:1089C000298918A000F028FDFEBD00000D930008C5
:1089D0004C000020004F0008C4000020440D00207F
:1089E00000000020666666666666E63F0000084096
:1089F000F853E3A59B843E40FF7F0000C81400208D
:108A0000B1EAC7A949443A202564202E0D0A000086
:108A1000CDA8D1B6BCE4B8F43A202564206D732EFD
:108A20000D0A0000B5A5B4CECDA8D1B6BBF9D5BE10
:108A3000CAFDC1BF3A202564B8F62E0D0A00000019
:108A400070B586B014216846FCF7B1FB01250F4EC6
:108A5000ED03002229463046FEF725F901200024C7
:108A6000019002946946009503943046FEF75AF847
:108A70000320019002946946009503943046FEF766
:108A800051F8022000F0DEFE06B070BD0004005078
:108A90000088704770470000F8B5044600206A4619
:108AA0001080194D55222A70AA226A700322AA70DA
:108AB000661DEE702A716971144A49008918AC71FB
:108AC0002246E81DFCF75AFB002007E029186A46F9
:108AD0008978128889186A461180401CB042F5DBFB
:108AE000611DA81CFDF742F801466846018029195E
:108AF0000078C871684640780872214609310248FA
:108B000000F064FAF8BD000008140020440D0020B5
:108B100070B50F48C088FCF7E5FD0E4A0E4BFCF718
:108B2000E5FC0E4E04460D467089FCF7DBFD22463F
:108B30002B46FCF729FCFCF7F7FD094A510C00E035
:108B400080188842FCDC074970810968486170BD63
:108B5000440D0020FCA9F1D24D624040C400002029
:108B60000180FFFFC8140020034A1168382389B22E
:108B700099430143116070470030014010B5FEF782
:108B80009FF810BD10B59AB034216846FCF70FFB72
:108B900014210DA8FCF70BFB1C2112A8FCF707FB06
:108BA0001B4801680324E402A143C2148918016030
:108BB000FEF736FA17480169A143016106200090CB
:108BC000FF20013002900120039010200490022029
:108BD000099040040B90000100240C900A94684610
:108BE000FEF7EAFB0F200D9003200E900F941094D7
:108BF000012111940DA8FEF7CDFA812012900320D7
:108C000080041890149412A8FEF712FA1AB010BD3E
:108C10000070004040100240104801688215114366
:108C20000160C1680E4A1140C16001680D4A1140DF
:108C3000016081684908490081600168012292044D
:108C400091430160C168FD2212049143C16000217B
:108C50000161064904488860704700000010024026
:108C60000C40FF88F6FFF6FE0050000800ED00E023
:108C700070B501F05FF80F4C0F4D606402E001F039
:108C800059F86064A842FAD10020E08220780028D8
:108C900009D0012802D0022805D102E0FDF706F92B
:108CA00001E0FFF74BFA00F037FFFDF7CBF903497E
:108CB000087070BD500000203001CADEC4000020E2
:108CC00010B5818CC90707D001684A6801235B048D
:108CD0009A43836A1A434A60818C890707D50168E1
:108CE0004A6801231B049A43C36A1A434A60818C71
:108CF000490707D501684A6801239B049A43036B1F
:108D00001A434A60818C090707D501684A68012324
:108D1000DB039A43436B1A434A60818CC90607D52B
:108D20000268916801231B039943836B1943916087
:108D3000818C890607D501688A6801235B039A4301
:108D4000C36B1A438A60818C490612D503685A683E
:108D500001210905046C8A4322435A60026C8A424D
:108D600007D10268516803235B059943436C19439B
:108D70005160818C090607D501684A680123DB042C
:108D8000806C9A4302434A6010BD0000F8B500268B
:108D90000446C667FDF78EFF054620680068124F3F
:108DA000000709D501212B460022490520460097DE
:108DB00000F052FA00280DD12068006840070BD55A
:108DC00001212B46002289052046009700F044FA35
:108DD000002801D00320F8BD20206067A067603420
:108DE00026740020F8BD0000FFFFFF01F8B5174C06
:108DF000C826E078002828D16079002825D10120F4
:108E00006071134D686B002700281DD0686BC82166
:108E1000081A14E00F48E168405C616988470E4811
:108E20000E49008840000880E068401CE060E0686F
:108E3000C82800DBE760696BC820401A761EE1682D
:108E4000814201D0002EE5DC6771F8BD38000020BA
:108E5000000002407C0C0020D8000020E800002028
:108E600070B5224CE07800283FD1207900283CD111
:108E7000012020711E4EF16900250906002933DA10
:108E80002156625791420AD1F06940062CD5A0794B
:108E9000002829D0A5712089401C208124E0A179D7
:108EA000002903D1A0710A2000F0D3FC0020205635
:108EB000CC2148430F494218206912181279B26236
:108EC000401C00222061A256CC235A43895881427B
:108ED0000ADC25612078401C207020780E2800D103
:108EE0002570A078401CA070257170BD380000204E
:108EF000003801405401002010B5806A002201466C
:108F000040314A834A82FEF7EAFC10BD70B5846A9C
:108F1000606FA56F2168896800260906002906DAB6
:108F2000212804D152200653204600F047F820683B
:108F30008068400606D5222D04D15A2006532046CB
:108F400000F02CF8E06F10210843E0672046FEF7A0
:108F5000C6FC70BD10B501460968806A09688906BB
:108F600014D400225A210A5201680A68FF230133EF
:108F70009A430A6001688A68520852008A60016850
:108F80008A6840239A438A6020218167FEF742FE67
:108F900010BD10B5806AFEF73EFE10BD01680A687C
:108FA000FF2321339A430A6001688A6852085200FD
:108FB0008A602021816700210166704701680A6884
:108FC000C0239A430A6020214167704770B5164C50
:108FD000E278002A0CD12279002A09D10122E2701C
:108FE0000025C82903DC0222A256002A01DCE57014
:108FF00070BD0123E356CC2253430C4AD1500123C8
:10900000E356CC2673439B180A460146181DFCF70D
:10901000B5F86078401C607060780E2800D16570EB
:10902000A078401EA070E2E7380000205401002024
:10903000F8B504462669A268E769324366691020DC
:1090400000253E432368324378491E68784F3E40EE
:1090500016431E6023685A6803263603B243E66847
:1090600032435A602368A2698B4201D0266A324398
:109070009E680B273F02BE4316439E606D4E2368D9
:109080006D4AB3420CD1D2689207920F06D0012AE2
:1090900038D0022A34D0032A20D11EE001201DE05E
:1090A000664EB3420AD1D2680C26324026D0042A3A
:1090B00028D0082A24D00C2A10D10EE08B420DD1E2
:1090C000D66803229202164018D001229202B61AE4
:1090D00018D0B61A14D0964200D10820564A01265C
:1090E000403A574FF6038B4236D100280CD0022865
:1090F0000DD0042812D008281FD11CE00020EDE775
:109100000220EBE70420E9E7FEF7FAF808E0106830
:10911000C00601D5384605E04A4803E0FEF710F9DD
:10912000002873D0626851005118814205D811039C
:10913000814202D303E03046F4E7012566E0010EE8
:1091400006025008002330185941FBF7E7FF0321BE
:109150000902411A3C4A55E0E169B14232D10300AB
:1091600000F081F909070A0D06250606062B060000
:10917000E3E7FEF7C5F81CE0FEF7D2F819E0106847
:109180006168C00602D54808304A01E0304A480804
:109190008018FBF7ADFF80B201462E4A103991428C
:1091A000CBD8511C01400007400F08432CE0FEF7CC
:1091B000C7F8616840004A08EAE761680122480888
:1091C0001204E5E7030000F04EF909070A0D062630
:1091D0000606062C0600B0E7FEF792F81DE0FEF743
:1091E0009FF81AE010686168C00602D54808C019E7
:1091F00002E014484A081018FBF77AFF80B20146D3
:10920000144A1039914298D82168C860002020661D
:1092100060662846F8BDFEF793F861684A08801832
:10922000EAE7616848088019E6E700000048004066
:10923000F369FFEF00380140401002400044004055
:1092400000093D000024F400FFFC0F0000127A002A
:109250000048E801EFFF0000FFB581B017460E4659
:1092600004460A9D09E0681C07D0FDF723FD049918
:10927000401AA8420CD8002D0AD02068C169304697
:10928000884318D00020B842EDD0002005B0F0BDD2
:1092900020680168FF22A132914301602068816843
:1092A00049084900816020206067A0670020603481
:1092B00020740320EAE70120E5E7000010B5044927
:1092C0001020096808620248FEF70AFB10BD000082
:1092D0008C15002001490D2088707047380000204F
:1092E00010B50748818A49008184FEF7E5FDFEF745
:1092F000BDFEC82203490448FEF730FC10BD000043
:10930000C40000207C0C00208C150020F8B53D4CDA
:10931000002321783C4A1D46082910D0072945D052
:1093200006294ED0052950D0042951D0032952D006
:10933000002954D0012956D0022958D059E0A178EB
:1093400000264A1F04E0304FBF5DFB189BB2761C1D
:109350009642F8DB667927799A195118E378627892
:10936000C9188918C9194018C0071AD0012E14D07D
:10937000022E16D125482449C018FBF7FFFE00F045
:109380005DFF642000F05EFABFF34F8F2149204853
:10939000C860BFF34F8F00BFFDE759081046FFF7C5
:1093A0007BFB2570E570A570A571F8BDA1795054BF
:1093B000491CC8B2A071A178491F8842F5D1082084
:1093C00001E0607007202070F8BDE0700620FAE729
:1093D00060710520F7E7A070E5700420F3E75528D9
:1093E00007D10120EFE7AA2803D10220EBE70328E9
:1093F00003D02570E570A570F8BD032020702071A2
:10940000F8BD0000BB000020A4130020440D002084
:109410000400FA0500ED00E00FB410B503A9044BF9
:10942000044A029800F002F910BC08BC04B01847C6
:1094300075A00008140100202021020C01D0102189
:109440001046020A01D010460839020901D0104620
:10945000091F820801D01046891E420801D0881ECB
:109460007047081A704730B47446641E2578641C2F
:10947000AB4200D21D46635D5B00E31830BC184769
:1094800002E008C8121F08C1002AFAD170477047CD
:10949000002001E001C1121F002AFBD1704708B56E
:1094A0000021684601706B46012202212C2000F049
:1094B00081FD0221684601706B4601222C2000F0DC
:1094C00079FD08BD38B504466D20694608706B46C5
:1094D000012207492E2000F06DFD0649002C01D025
:1094E000054A00E0054A2E2000F04AFD38BD000084
:1094F0000608000006180000070600000716000016
:1095000038B504466B4602220021362000F018FCD4
:10951000B3212300FFF7A7FF0E0F08153A3A3A3A96
:109520001C273A3A2F34483A0021684601704078A7
:109530004108490014E06946087880088000401C12
:1095400004E06946087880088000801C08701DE0EF
:10955000684602780A404832027041788020014310
:109560006846417012E0684602780A40027040780E
:109570004106490EF4E7694648780221084303E0B2
:1095800069464878FD210840694648706B460122CB
:109590000021362000F00EFD012200AB11463620DE
:1095A000013300F007FD38BD69460878CF21084037
:1095B00069462030CAE708B5032168464170012199
:1095C00001706B4602220021362000F0F3FC0122DC
:1095D000D20306212D2000F0D3FC012000F032F947
:1095E0000120FFF78DFF08BD08B5020A69464A70E1
:1095F00008706B46022204212D2000F0DBFC0320C2
:10960000694608706B46012206212D2000F0D2FC2D
:109610000020694608706B46012206212D2000F0CB
:10962000C9FC0A212D2000F071FB08BDFFB58DB0EB
:109630000446002506E025280AD0109A0F99904785
:10964000641C6D1C20780028F5D1284611B0F0BDAF
:1096500000270121484A009700E00743641C237853
:109660000846203B98401042F7D120782E2817D189
:10967000042007436078641C2A280CD10E98641CCF
:1096800002C800910E900BE000990A225143303934
:109690004018641C00902078014630390929F3D91C
:1096A00020780028D1D0642808D0692806D07528F1
:1096B0001ED0109A0F9990476D1C5BE00A200E99FE
:1096C000019001C90E91002802DA40422D2102E0EA
:1096D000390504D52B216A461172012103E0F907EF
:1096E00004D02021F7E70BAE0B910DE00021FAE743
:1096F0000A200E99019001C90E91F7E70199FBF735
:10970000F7FC3031761E31700028F7D103A8801B9A
:1097100020300190780701D5009801E001200090E9
:109720000199884201DD401A00E0002000270090E6
:1097300006E002A8109AC05D0F9990476D1C7F1C2F
:109740000B988742F5DB04E0109A30200F99904780
:109750006D1C0099481E00900029F5DC05E030786A
:10976000109A761C0F9990476D1C0199481E019024
:109770000029F4DC641C65E709280100F8B54A00FB
:109780002B4B520DD6182B4A0C460546142E2BDABD
:10979000002E12DA284BFBF7F7FD00221346FCF7E8
:1097A00009F940D2002C03DA0124E40700253AE04D
:1097B0002046284337D0214C14E0214F0B46F74078
:1097C0003B402B4331D01C4BFBF7DEFD0022134600
:1097D000FCF7F0F827D2002C03DD01200005F04053
:1097E0000419BC4300251EE0332E1EDC334600273F
:1097F000143BFF43DF40384217D00F4BFBF76EFEA0
:1098000000221346FCF7D6F80DD2002C0ADD142EE8
:109810000CD03420811B012088404019A84200D27E
:10982000641C0546BD4321462846F8BD641CF9E783
:1098300001FCFFFF9C7500883CE4377E0000F03F90
:10984000FFFF0F007D2110B5C900484300F001F86B
:1098500010BD002140E000BF00BF00BF00BF00BF3F
:1098600000BF00BF00BF00BF00BF00BF00BF00BF00
:1098700000BF00BF00BF00BF00BF00BF00BF00BFF0
:1098800000BF00BF00BF00BF00BF00BF00BF00BFE0
:1098900000BF00BF00BF00BF00BF00BF00BF00BFD0
:1098A00000BF00BF00BF00BF00BF00BF00BF00BFC0
:1098B00000BF00BF00BF00BF00BF00BF00BF00BFB0
:1098C00000BF00BF00BF00BF00BF00BF00BF00BFA0
:1098D00000BF00BF00BF491C8142BCD370470000DD
:1098E000FEB5044600200190009060797349400065
:1098F0000E5A61782578491E7148CFB20163042D54
:1099000077D0072D75D000210291217801736C4921
:10991000E379012292058969002B6CD09143816122
:109920006748217A4173217A82698907890B0A4342
:1099300082610021042000F02EFB324661492E2076
:1099400000F01EFB3846FFF7BDFD5F4E0522705D3F
:10995000810040185D49431807212B2000F02AFBA5
:109960005B49029801220B180B21282000F022FBF2
:10997000705D584980000A580C21282000F00BFB2C
:10998000E079554980004018A1794900425A0221E6
:10999000272000F0F5FA51487E00825B0421272041
:1099A00000F0EEFAE079002829D0A07804282CD025
:1099B00028206946087220220621272000F0E0FABC
:1099C00002AB01222621272000F0F4FA4449380195
:1099D0004018E178890042580821272000F0DBFA7E
:1099E000A17A601C627A0902114313D016E000E0EC
:1099F00001E0012188E71143F608816190E76422C4
:109A00000621272000F0BCFAE0E710206946087222
:109A10000246D1E733490172090A4172417A007A5C
:109A20000A0202432021272000F0AAFA2E4F0C211F
:109A300023203A6800F0AFFAF0198288042123202D
:109A400000F09EFAA07900280BD0E0792749012286
:109A500043180021212000F0ADFA032001900120DD
:109A600000902A07120F100102436078002180073E
:109A7000000B024301980005024300984004024392
:109A80002079C006400902436079C00602431F20C6
:109A900000F081FAA07861780123084302040848A5
:109AA000DB030261E179490319430A4302610021A2
:109AB000082000F070FA0020FEBD000008A3000896
:109AC0001801002004280000B0A2000801000020B6
:109AD0001F000020B8A20008D8A20008E4A20008D5
:109AE000E8A2000841100000D0A2000821000020D8
:109AF00038B50C4607498A8B002102432C2000F020
:109B00003FFA684604706B46012206212C2000F0C3
:109B100051FA38BD1801002010B5FFF7C0FC10BD88
:109B200010B504460421362000F0F0F80121C902E6
:109B3000002C01D0084300E088430246042136206F
:109B400000F029FA10BD000038B5402069460870C1
:109B500000210E2000F0DAF80446002211460E2003
:109B600000F019FA6B46012200210D2000F022FAC4
:109B7000074A00210F2000F00EFA00F0E7F9224614
:109B800000210E2000F007FA02480021017338BDC1
:109B9000F8FF2724380100207CB5054604206946DB
:109BA00008704B4C002060752146203120634871BD
:109BB0000873A0836063A06300F0BCF8454E20608A
:109BC00002E000F0B7F82060B042FAD10020FFF7C1
:109BD00097FC41480078242801D9243806E0062162
:109BE000FBF786FA0622101A400108430206010418
:109BF0000A4301020A43024300211E2000F0CBF970
:109C00006B4601220021242000F0D4F91E20FFF72A
:109C1000EBFC86B2300AA0730420FFF7E5FC0006D7
:109C2000000E0DD002206946087101AB01221221FD
:109C30002D2000F0BFF9A08B012109030843A08368
:109C400000F078F820600620FFF7CEFC6060072067
:109C5000FFF7CAFCA060F006C00E207501D11020ED
:109C60002075C0B200F0E2F9E80707D0FFF7A3FCC7
:109C7000A08B0121C9020843A0830AE005213620F8
:109C800000F02EF81549084002460521362000F064
:109C900077F90120FFF734FC0021042000F036F8AA
:109CA000A0610021262000F031F815218903084326
:109CB00002460021262000F06EF9002226213620DF
:109CC00000F05EF900F036F8206000207CBD000056
:109CD000180100203001CADE00000020FFFD000056
:109CE00038B5094C89B280B26B46022200F028F8E0
:109CF000002806D1684640780102684600780818B6
:109D000084B2204638BD0000FFFF000038B50024B3
:109D1000E44389B280B26B46042200F011F80028B7
:109D200006D103216846435C2202D418491EFAD5A5
:109D3000204638BD10B500210846FFF7E7FF10BDEB
:109D400038B5002909D0402420436C462070C8B2A1
:109D50007F2906D8607002200AE069460870012059
:109D600006E0802420436C466070C809A070032080
:109D7000694600F03DFA38BD10B5144603460A4660
:109D800021461120FFF7DCFF10BD10B50346052268
:109D900000211520FFF7D4FF10BD10B501210620CA
:109DA000FFF7B4FF10BD10B50346052200211720B0
:109DB000FFF7C6FF10BD38B505460020694608709C
:109DC00000F0C4F8FF2401342246002D01D0032204
:109DD000120200210D2000F0D3F8002D13D06B46A5
:109DE000012203210F20FFF7ABFF68460078000730
:109DF00009D5FFF7A9FE224600210D2000F0C0F88A
:109E00000020C04338BD002038BD10B502460121F6
:109E10000A2000F0C0F810BD10B5044600211A2039
:109E2000FFF774FF000D22030005120B024300210F
:109E30001A2000F0B0F810BD10B5024602492E20DD
:109E400000F09EF810BD000004180000F8B50546AB
:109E50006B46012203210420FFF772FF0126114CFB
:109E60003607002D0DD02A4600210C2000F088F87E
:109E7000694608781021084369460870A069304394
:109E800007E069460878EF21084069460870A06934
:109E9000B0430B46A06101220321042000F08AF8A0
:109EA000F8BD00001801002010B50246002118205E
:109EB00000F066F810BD0000F8B5074600256846BA
:109EC0000570B807204C2E4600280ADA8020694623
:109ED00008706B46012200210D2000F06BF8012074
:109EE0002073F8076946087821D00621084369469F
:109EF00008706B46012200210D2000F05BF8032161
:109F00000F20FFF7EDFE8121C900084219D0402043
:109F1000694608706B46012200210D2000F04AF8C6
:109F20000020FFF7FDFD00252673ED4309E0022127
:109F30000843694608706B46012200210D2000F09D
:109F400039F82846F8BD0000380100201CB56B46E2
:109F5000012203210F20FFF7F3FE6846007840221C
:109F6000C1091040C9014000814208D00120694662
:109F70000871024601AB03210D2000F01BF81CBD47
:109F800008B56B461A70120A5A7089B280B2022262
:109F900000F010F808BD38B500236C46E254120AF0
:109FA0005B1C042BFADB89B280B22346042200F04A
:109FB00001F838BD38B58024002909D0C0252843D0
:109FC0006D462870C8B27F2907D86870022009E062
:109FD000204369460870012004E020436870C809E6
:109FE000A8700320694600F03FF938BD10B514464B
:109FF000012312189B029A4202D90020C04310BDCF
:10A000000B46821E21460920FFF7D4FF002010BD19
:10A0100010B5054A8905126901430A430021082049
:10A02000FFF7B9FF002010BD1801002038B5044625
:10A030006B4601220E212B20FFF782FE6846007836
:10A04000E10640094001C90E0143684601706B46B4
:10A0500001220E212B20FFF7ADFF38BD10B50021E6
:10A0600042541C06120A22431B0A491C0429F7DB2E
:10A0700010BD000013B501231A4669460248FDF7DA
:10A08000CBFD00981CBD00008C150020FCF720FEC5
:10A09000FEF778FDFDF724FF32493348002522C042
:10A0A00005608561C56131490562C1600838FCF70A
:10A0B00009FFFDF701FFFDF7D9FFFDF7B5FF052407
:10A0C00001222407D1032046FCF7EDFDFEF7F6FB45
:10A0D000FBF7A2FDFBF77AFD0721A015FFF708FDAE
:10A0E000FFF71AFD0122170339462046FCF7DBFD76
:10A0F0001D48C8221E49C430FDF730FD7D200001F7
:10A10000FCF7ECFB1B4E1C4C2079002827D0207A52
:10A11000002824D0FEF736FD257120780F2809D9B4
:10A12000012239463046FCF7BEFDFEF7A1FD0022B4
:10A13000394609E0012251033046FCF7B4FDFEF731
:10A1400097FD0022012149033046FCF7ACFDFDF7E5
:10A15000D3FDA08C0028D7D0401EA084D4E7FDF703
:10A16000CBFDD1E7007C0040C8140020FFFF0000B9
:10A170007C0C002000040050C400002010B5012217
:10A18000920218491848FBF7BBFD16481749028888
:10A190008A4226D0018004218180FF21F531C180CF
:10A1A0000A21018100211E224181D24382810122A4
:10A1B000C2810184018241828182C18201838183C3
:10A1C0004323C38602230387782343878287C2877A
:10A1D000024640329180118451849184C18300F001
:10A1E0002DF810BD440D002000FC0008AA55000009
:10A1F000F0B58C4600251026052109078E620E4C0D
:10A2000008E067467F5DE760A768FF07FCD0E76866
:10A210001F706D1C8542F4DB0020074606E0E760F6
:10A22000A568ED07FCD0E5681D54401C9042F6D3AC
:10A230008E610020F0BD00000030014070B572B6A4
:10A240000124074DA40221462846FBF73FFD0028C4
:10A2500004D0224603492846FBF7DCFD62B670BDF8
:10A2600000FC0008440D0020F0B50025102605274D
:10A270009C463F070B46BE620C4C06E0595DE16010
:10A28000A168C907FCD0E1686D1C8542F6DB00209F
:10A2900007E06146095CE160A168C907FCD0E1689C
:10A2A000401C9042F5D3BE610020F0BD003001405B
:10A2B0000000010203040005405C0000A05C0400F3
:10A2C000C06C0800805C0400E03F1E00E07D1E00C2
:10A2D00007A9022570889B880A0016000100060065
:10A2E0000100020087008D002D001A3152001A3340
:10A2F0009A001A351D011A376B003B31BE003B3303
:10A300005E013B3596023B37000099599959EB5154
:10A310008F421E45142E0080EB51F5283333E13A6D
:10A32000703DE13AC235852BC2353333C235C23573
:10A33000AE47E13A5138A330513800C1814001C0E5
:10A34000804101C0804100C1814001C0804100C105
:10A35000814000C1814001C0804101C0804100C1F5
:10A36000814000C1814001C0804100C1814001C0E5
:10A37000804101C0804100C1814001C0804100C1D5
:10A38000814000C1814001C0804100C1814001C0C5
:10A39000804101C0804100C1814000C1814001C0B5
:10A3A000804101C0804100C1814001C0804100C1A5
:10A3B000814000C1814001C0804101C0804100C195
:10A3C000814000C1814001C0804100C1814001C085
:10A3D000804101C0804100C1814000C1814001C075
:10A3E000804101C0804100C1814001C0804100C165
:10A3F000814000C1814001C0804100C1814001C055
:10A40000804101C0804100C1814001C0804100C144
:10A41000814000C1814001C0804101C0804100C134
:10A42000814000C1814001C0804100C1814001C024
:10A43000804101C0804100C1814000C0C101C3030F
:10A4400002C2C60607C705C5C404CC0C0DCD0FCF8C
:10A45000CE0E0ACACB0BC90908C8D81819D91BDBFC
:10A46000DA1A1EDEDF1FDD1D1CDC14D4D515D7174C
:10A4700016D6D21213D311D1D010F03031F133F3FC
:10A48000F23236F6F737F53534F43CFCFD3DFF3F4C
:10A490003EFEFA3A3BFB39F9F83828E8E929EB2B7C
:10A4A0002AEAEE2E2FEF2DEDEC2CE42425E527E70C
:10A4B000E62622E2E323E12120E0A06061A163A37C
:10A4C000A26266A6A767A56564A46CACAD6DAF6F0C
:10A4D0006EAEAA6A6BAB69A9A86878B8B979BB7B7C
:10A4E0007ABABE7E7FBF7DBDBC7CB47475B577B7CC
:10A4F000B67672B2B373B17170B0509091519353FC
:10A50000529296565797559594549C5C5D9D5F9FCB
:10A510009E5E5A9A9B5B99595898884849894B8BFB
:10A520008A4A4E8E8F4F8D4D4C8C4484854587478B
:10A530004686824243834181804000000000000043
:10A5400000000102030406070809030406080C10B2
:10A550001820300000000001020304007CA5000860
:10A5600000000020180100008094000894A6000854
:10A5700018010020A01900009094000800070400B2
:10A58000091E08054008260910400856080540081D
:10A59000261D040008BE1D040008BED8BC401008DB
:10A5A00001010000000000000000C8420000C84295
:10A5B000000000000000000000000000000000009B
:10A5C0000000000000000000000000000200000089
:10A5D000000000000000000000000000000000007B
:10A5E0008C0A0000000000000000000000000000D5
:10A5F000000000000000000000000000000000005B
:10A60000000000000000000000000000000000004A
:10A61000000000000000000000000000000000003A
:10A62000000000000000000000000000050214000F
:10A630000909010200810000000000000100000083
:10A640000001000000000000000000000000000009
:10A6500000000000000000000000000000000000FA
:10A6600000000000000000000000C84200000000E0
:10A6700000000000000000000000000000000000DA
:10A6800000000000000000000000000000002000AA
:04A6900000000000C6
:04000005080050C1DE
:00000001FF
